:0A00000075817F7401F58F02002E58
:10002B000241B8C294D294C2A4D2A57532007533E2
:10003B000075340075350075360075370075630033
:10004B00756600756700756400754500754601752A
:10005B00470175600175610175620175480075494D
:10006B0000754A00754B00754C01C233754D007518
:10007B005A00755900755C00755B0075530075541B
:10008B00007552F0754E00754F00755000755D0090
:10009B00C20AC22EC20CC210C211C214C215C212A5
:1000AB00C213C20FC216C217C218C219C21AC21B80
:1000BB00C21CC21DC21EC21FC220D209C234C2350D
:1000CB00D2367400900030F0900031F0900032F096
:1000DB00900033F0900034F07400900035F09000F5
:1000EB0036F090027F7400F0A37404F0A37407F051
:1000FB00A37409F09001207416F09001217438F06C
:10010B0012395012395C9001177401F0900122746E
:10011B0001F09001237401F09001277401F090011C
:10012B00187401F09001247401F09001197401F01E
:10013B0090011A7401F090011B7401F090011F746F
:10014B0001F090011C7401F090011D7401F09001FD
:10015B001E7401F09001297401F0753C00753D008F
:10016B001209557538001204DF1203801204EC7566
:10017B003800120203124192120751C2A1120AC196
:10018B00120ACB120AD5120AF3120B81120B9F1211
:10019B0004C51204DF120203120203753C30753DD5
:1001AB0008123EFC753C00753D00123E9712415201
:1001BB00121DE5121EA012248BC202C2031232ECD6
:1001CB001220BC12391812327C1235A712211B9047
:1001DB000122E0B403061233A80201EC50F81225F9
:1001EB002A121CBD12201B12246C0201D178327909
:1001FB00FF0000D9FCD8F822786479FF0000D9FC05
:10020B00D8F82278967996D9FED8FA2278FF799B7E
:10021B00D9FED8FA22780A790AD9FED8FA22E6272B
:10022B00F5270809E637F528782722C3E697F5273F
:10023B000809E697F5287827228627872908098653
:10024B0028872A1202C9782C22862C08862D08862C
:10025B002E08862F872909872A12026C7827792E78
:10026B00227530007531101202AE12027F1202A2FB
:10027B00D531F422C3E52E9529E52F952AE5309447
:10028B0000500122E52E9529F52EE52F952AF52F05
:10029B00E5309400F53022B3E52733F527E5283315
:1002AB00F52822C3E52C33F52CE52D33F52DE52E62
:1002BB0033F52EE52F33F52FE53033F53022E527D7
:1002CB008529F0A4F52C85F02DE528852AF0A4F5D9
:0C02DB002E85F02FE5288529F0A4252DA4
:1002E700F52DE52E35F0F52EE52F3400F52FE52712
:1002F700852AF0A4252DF52DE52E35F0F52EE52FD1
:100307003400F52F22E538B4101120010ED201C2B6
:100317008174C0120350D282C28222E538B4200F02
:10032700C2817480120350D282C28275380022C201
:1003370001A2009281900000E5822538F582E01243
:100347000350D282C282053822F954F053800F42FB
:1003570080D282C282E9C454F053800F42802212B5
:1003670002032212020312020312020312020312F1
:10037700020312020312020322C28212036612034D
:1003870066C281C283120203D282C287C286D28525
:10039700D284120203C282120366C281C28312028E
:1003A70003D282C287C286D285D284120203C28256
:1003B700120366C281C283120203D282C287C28637
:1003C700D285D284120203C282120366C281C2831B
:1003D700120203D282C287C286D285C28412020366
:1003E700C282120366C281C283120203D282C2870B
:1003F700C286D285C284120203C282120366C281F8
:10040700C283120203D282D287C286C285C28412F5
:100417000203C282120366C281C283120203D2821E
:10042700C287C286C285C284120203C282120366D1
:10043700C281C283120203D282D287D286D285C2F8
:1004470084120203C282120366C281C283120203AC
:10045700D282C287C286C285C284120203C28212B6
:100467000366C281C283120203D282C287C286C2D6
:1004770085D284120203C282120366C281C283122A
:100487000203D282C287C286C285C284120203C215
:1004970082120366C281C283120203D282C287D24A
:1004A70086D285C284120203C282120366D2002258
:1004B70005A2E493A305A2F0A3DBF505A222900F02
:1004C7006F05A29000007B200204B7900F8F05A252
:1004D7009000007B200204B7900FDF05A290000078
:1004E7007B200204B7C283C2817440120350D282B8
:1004F700C282120217D2817400120350D282C282C2
:10050700120217D281741E120350D282C2821202C3
:1005170017D281741E120350D282C282120217D2DE
:1005270081741E120350D282C282120217D28174C2
:100537001E120350D282C282120217D281741E1277
:100547000350D282C282120217D281741E12035044
:10055700D282C282120217C283C281744812035028
:10056700D282C282120217D2817404120350D2823D
:10057700C282120217D281740E120350D282C28233
:10058700120217D2817415120350D282C28212024C
:1005970017D2817404120350D282C282120217D278
:1005A700817404120350D282C282120217D281745C
:1005B70004120350D282C282120217D2817404122B
:1005C7000350D282C282120217D2817400120350E2
:1005D700D282C282120217C283C2817450120350A0
:1005E700D282C282120217D2817404120350D282BD
:1005F700C282120217D2817404120350D282C282BD
:10060700120217D2817404120350D282C2821202DC
:1006170017D2817404120350D282C282120217D2F7
:10062700817415120350D282C282120217D28174CA
:100637000E120350D282C282120217D281740412A0
:100647000350D282C282120217D281740012035061
:0E065700D282C282120217C283C2817458126C
:100665000350D282C282120217D28174041203503F
:10067500D282C282120217D281740E120350D28224
:10068500C282120217D2817415120350D282C2821D
:10069500120217D2817404120350D282C28212024E
:1006A50017D2817415120350D282C282120217D258
:1006B50081740E120350D282C282120217D2817443
:1006C50004120350D282C282120217D28174001220
:1006D5000350D282C282120217222430F02275F012
:1006E5000A84AFF075F00A84E5F02430F0EF243089
:1006F500A3F02275F00A84AFF075F00A842430F077
:10070500E5F02430A3F0EF2430A3F0221206F8A37D
:10071500742CF0EE2430A3F022D281C2831202039E
:10072500D282D287D286D285D284120203C28212A5
:100735000366D281C283120203D282D287D286D2C5
:1007450085D284120203C282120366221204DF12CA
:10075500020312020312020312020312020312021F
:10076500031202031204C5753C24753D00120203F1
:10077500120203753C30753D001202031202037527
:100785003C20753D02120203120203753C20753DA3
:1007950008120203120203753C20753D2012020364
:1007A500120203753C20753D801202031202037587
:1007B5003C20753D10120203120203753C20753D65
:1007C50004120203120203753CA0753D00120203D8
:1007D500120203753C60753D001202031202037597
:1007E5003C28753D00120203120203753C22753D3B
:1007F50000120203120203753C20753D001202032C
:10080500120203753C20753D0012020312020375A6
:100815003C20753D40120203120203753C21753DD3
:1008250000120203120203753C20753D01120203FA
:10083500120203753C20753D001204D21202031208
:10084500020312020312020312020312020312022E
:10085500031202031202031202031202031202031D
:1008650012020312020312020312020312020312FE
:1008750002031202031202031204DF120203120220
:1008850003120203120203221202031202031202CE
:1008950003120203120203120203120203120203DD
:1008A50012020312020312020312020312020312BE
:1008B50002031202031202031202031202031202BE
:1008C50003120203120203120203120203120203AD
:1008D500120203120203120203120203120203128E
:1008E500020312020312020312020312020312028E
:1008F500031202031202031202031202031202037D
:100905002220B2047539002220B103D204227539A0
:100915000122E539B53A0485393A22B40019200493
:100925000A053B85393AD206D20222153BC2048517
:10093500393AD206D2032220040A153B85393AD228
:1009450006D20322053BC20485393AD206D20222D9
:10095500C2B3C2B4C2B5E53CF4200E0244FE7F0822
:100965003392B6D2B5C2B5DFF7B2B30000C2B3E574
:100975003DF4200E0244FE79083392B6C2B5D2B5D5
:10098500D9F7D2B40000C2B422C293D2937908C277
:1009950090A29133D290D9F7F53EC293D2937908BC
:1009A500C290A29233D290D9F7F53F22E582C45482
:1009B5000FF9E583C46922E5820303543FF9E58312
:1009C500030354C069227A0CC2A6D2A3A2C133C9BB
:0E09D50033C9C2A3DAF2F8D2A622C2A3C2A688
:1009E3003392A7D2A3DAF5C2A31209CBE95403F9D0
:1009F300227A0574C01209DFF5838882227A05748E
:100A0300C81209DFF5838882227A0574D01209DFC0
:100A1300F5838882227A0574D81209DFF5838882E8
:100A230022858232858333753400753500783275BB
:100A33003678753700793612024485523675370396
:100A43007936120254E62285823285833375340067
:100A530075350078327536047537007936120229F8
:100A6300863208863375340075350078327536E87A
:100A73007537037936120244753655753721793641
:100A8300120254E62285823285833375340075352C
:100A93000078327536117537007936120254E62222
:100AA30022C2A0E8120AB5E9120AB5EA120AB5D2BF
:100AB300A0227B08D2A13392A2C2A1DBF722784005
:100AC300790F7A00120AA4227869790F7A00120A40
:100AD300A422787779007A00120AA422782F79FF6A
:100AE3007AF0120AA422782F79807A00120AA422BB
:100AF300782F79007A00120AA422782FF97A00124B
:100B03000AA422782F791F7A80120AA422782F79D7
:100B13003F7A00120AA422782F79FC7A00120AA4E1
:100B230022E583C454F0F9E582C4FA540F49F9EA83
:100B330054F0FA22120B247800120AA422120B2476
:100B43007801120AA422120B247802120AA4221298
:100B53000B247803120AA422120B2478A0120B642C
:100B630022C296E8120B75E9120B75EA120B75D2C5
:100B730096227B08D2A1339295C2A1DBF722782774
:100B830079007A00120B642278A079FF7AF0120BB5
:100B9300642278A079807A00120B642278A079000D
:100BA3007A00120B642278A0791F7A80120B6422D8
:100BB30078A0793F7A00120B642278A079FC7A003E
:100BC300120B6422F532753300783275362275378D
:100BD300007936120244868208868322F532753301
:100BE30000783275362275370079361202448682D0
:100BF30008868322120EA1F53275330078327536DA
:100C03002A7537007936120244868208868322F5D4
:100C13003275330078327536207537007936120213
:100C230044868208868322900030E004B410027464
:100C330000F0900020A98229F582E022900034E0A0
:100C4300FA900031E004B40F0274FFF0900F4F9359
:100C53002A900034F0900033E004B410027400F0E2
:100C6300F9900034E0FA900020E58229F582EAF059
:100C730022900034E0FA900032E004B4110274FFD1
:100C8300F0900F5E932A900034F0120C5822120C4D
:100C93002A54016008120C2A541F246022747F22F4
:100CA300F974FF89F084F5F0120C2A8422120C2ABD
:100CB30075F0208422120C2A75F033842401221249
:100CC3000C2A75F02084240122120C2A75F03F842B
:100CD300240122120C2A75F03384240322120C2AD5
:100CE30075F0108422120C2A75F01F8422120C2A2C
:100CF30075F02084F8120C2A75F03F842822120C18
:100D03002A540175F00CA422120C2A75F05584752F
:100D1300F00CA422B40101225003740122B4070190
:100D230022500122740722B40101225003740122CC
:100D3300B40A0122500122740A22B4010122500391
:100D4300740122B40D0122500122740D22B4010159
:0E0D5300225003740122B410012250012274B8
:100D61001022B40101225003740422B40401225060
:100D71000122740122B40101225003740A22B40A2F
:100D81000122500122740122B4010122500374187E
:100D910022B4180122500122740122B4010122500F
:100DA10003740122B43A0122500122743A22B4019F
:100DB10001225003740122B44801225001227448D7
:100DC10022B40101225003740022B44801225001CF
:100DD10022B4FF03740022744822B401012250039B
:100DE100740122B4040122500122740422B40101CD
:100DF100225003740122B4050122500122740522FC
:100E0100B40101225003740122B4200122500122B5
:100E1100742022B40101225003740122B402012280
:100E2100500122740222B40101225003740122B440
:100E3100020122500122740222B4010122500374E2
:100E41000122B4050122500122740522B4000122BD
:100E51005003740022B4050122500122740522B40A
:100E61000001225003740022B403012250012274B4
:100E71000322B4FF03740C22B40B0122500122742B
:100E81000C22B4FF02EC22B43C0122500122EC22DC
:100E9100B4FF03740022B40301225001227403221F
:100EA100B46001224002746022B4FF03740022B4D2
:100EB100240122500122742422B40101225003741E
:100EC1000122B4180122500122741822B401012216
:100ED1005003740122B4020122500122740222B48F
:100EE1000101225003740122B40201225001227433
:100EF1000222F990027AE0F55EE9B4010122500381
:100F0100740122B55E0122500122E55E22F99002B0
:100F11007AE0F55EE9B40101225003740122B55E65
:100F21000122500122740122B401012250037404F0
:100F310022B4040122500122740122B40101225081
:100F410003740122B40C0122500122740C22037F8C
:100F51002C0C0105712133E6FF0B576818BD09A65A
:100F61000D004B5D263585B196114093C8D32046BF
:100F710020204C20204120204D2020452020434886
:100F81004F5244204D414348494E452032202020B4
:100F910056455253494F4E20312E303620202020C5
:100FA100286329323031362D323031382020496ED4
:100FB100697420616C6C2044617461203F204F4B47
:100FC10020202020202020202020204E4F20205093
:100FD1006C65617365207761697420212020202070
:100FE1002020202020202020202020202020202000
:100FF10020202020202020202020202020204D4F94
:1010010044452050524F4752414D4D2020204D4FD5
:1010110044453C3E202343302020524F4F54202052
:101021005030312020234331202020202020202037
:10103100503031204449523A646F776E204449560A
:101041003A6E6F202023433120017363616C653A4E
:10105100503031202023433120027363616C653AA3
:10106100503031202023433120037363616C653A92
:1010710050303120202043484F52442020415250CB
:101081002F514152504547494F20205155414E540F
:10109100204C454E4748542053454C4543544C69D8
:1010A10073743A41303120202043484F52444C69F7
:1010B10073743A4130312020204152502F51202069
:1010C10041322020553031203C20326E643E3C6359
:0E10D100686F726420417270656767696F3ED8
:1010DF003C7363616C6520417270656767696F3E31
:1010EF003C737461626C2E5175616E74697A653EE2
:1010FF003C636C6F636B205175616E74697A653EEA
:10110F0063686F72647363616C6520757020646FC0
:10111F00776E616C7431616C743272616E646E6F74
:10112F0020202064697265637420706572204356B5
:10113F00202020207374657020627920737465708D
:10114F006F6666206F6E43484F5244202020202048
:10115F005343414C4520202020204B45594E4F549E
:10116F00453A20204C4953543A41303120205345C1
:10117F005455502020202020415250454747494F79
:10118F00202053415645202020202020726F6F745D
:10119F0020203173742020326E6420203374682035
:1011AF005452414E53504F53453A2020494E5055BB
:1011BF0054202020204F63746176652052616E6742
:1011CF00654F6374617665205472616E73706F73CF
:1011DF006520312D4F637420446972656374696FA4
:1011EF006E20322D4F637420446972656374696F8A
:1011FF006E20332D4F637420446972656374696F79
:10120F006E20202053455454494E475343484F5264
:10121F0044203E205530315343414C45203E20550C
:10122F0030312020204C495354203E2041507265CC
:10123F007373206B65792043484F5244212020530C
:10124F00544F52414745204F4B20212020205455C9
:10125F004E452D4D4F444520204155544F4C4F4145
:10126F0044206C617374207361766564204C6973DC
:10127F00742020202020202020204C6973743A20D5
:10128F00415365742043562D4F5554733A202B38D4
:10129F00564B45594E4F54453A2020432343204443
:1012AF0023442045204623462047234720412341FE
:1012BF002042030000000004000C000C03000C1877
:1012CF000C04000C182402000700070400070E1579
:1012DF0002000500050400050A0F020004000403C4
:1012EF000004080C0200030003030003060C0400B3
:1012FF0003070E0400030A11040003060A04000387
:10130F000A0E040003070B030003060C0400030777
:10131F000A0400030709030003070C030004070C6A
:10132F000400040709040004070A040004070B0360
:10133F000005070C030002070C040004090E03004C
:10134F0004080C030004060C040005070A0400043B
:10135F00080A040004060A0400040B0E0400040B20
:10136F000D0400040B0F040004070E04000B0E11F4
:10137F0004000B101504000B0E150400040B1203D0
:10138F0000000000202020202020202020554E4942
:10139F00534F4E4F202020202020204F43544156A2
:1013AF0045532031202020202020204F43544156E8
:1013BF0045532032202020202020204F43544156D7
:1013CF00455320332020202020202020204649462E
:1013DF00544820312020202020202020204649461C
:1013EF00544820322020202020202020464F5552C4
:1013FF00544820312020202020202020464F5552B5
:10140F005448203220202020205448495244206D37
:10141F00616A2031202020202020204155474D4552
:10142F004E54454420202020205448495244206DDA
:10143F00696E203120202020202044494D494E49FB
:0E144F005348454420202020204D494E4F5246
:10145D002061646420392020202020204D494E4FEA
:10146D005220372F31312020202020204D494E4F42
:10147D00522037206235202020202020204D494E3B
:10148D004F5220372F3920202020204D494E4F52CA
:10149D00206D616A203720202020202020204D49FA
:1014AD004E4F522062352020202020202020204D1C
:1014BD00494E4F5220372020202020202020204D23
:1014CD00494E4F5220362020202020202020202041
:1014DD00204D494E4F52202020202020202020201A
:1014ED00204D414A4F522020202020202020204DE9
:1014FD00414A4F5220362020202020202020204DF0
:10150D00414A4F52203720202020204D414A4F5232
:10151D00206D616A203720202020204D414A4F52F6
:10152D0020737573203420202020204D414A4F52C6
:10153D00207375732032202020202020204D414A19
:10154D004F5220362F3920202020202020204D41A1
:10155D004A4F5220233520202020202020204D418D
:10156D004A4F52206235202020202020204D414A14
:10157D004F5220372F342020202020204D414A4F1C
:10158D005220372023352020202020204D414A4F46
:10159D00522037206235202020202020204D414A26
:1015AD004F5220372F392020202020204D414A4FE7
:1015BD005220372062392020202020204D414A4FD3
:1015CD0052203720233920202020204D414A4F52D0
:1015DD00206164642039202020204D414A4F522043
:1015ED00372F392F31312020202020204D414A4FD7
:1015FD005220372F3133202020204D414A4F522089
:10160D00372F392F313320202020204D414A4F5282
:10161D00203762203131202020202020202020550D
:10162D004E49534F4E4F2020202020207573657258
:10163D002063686F726408000203050607080B003B
:10164D00000000060001040507080000000000006E
:10165D00050001030708000000000000000600035C
:10166D000407090A00000000000006000305060734
:10167D000A000000000000070001040507080B0028
:10168D00000000000C000102030405060708090A0A
:10169D000B05000204070900000000000000070010
:1016AD0001040507080B00000000000700010406F7
:1016BD00080A0B000000000005000205070A0000E3
:1016CD000000000000070002040507080A000000E2
:1016DD000000070003040607090A000000000007C8
:1016ED000002030607080B000000000005000203BE
:1016FD0007080000000000000005000105060A00B3
:10170D0000000000000005000105070800000000B2
:10171D0000000005000105070A00000000000000A0
:10172D0005000305070A0000000000000005000287
:10173D0005070A000000000000000500020407096B
:10174D0000000000000000070002040506080A0062
:10175D0000000000070001030406080A0000000055
:10176D0000070002040607080A0000000000070039
:10177D0002030507080B0000000000070001030528
:10178D0006090A0000000000070002040508090B05
:10179D000000000000070002030607090A00000010
:1017AD000000070001040507080A000000000007FB
:1017BD000003040607090B000000000007000103E9
:0E17CD000406080900000000000700020305E2
:1017DB0007090B0000000000070002040507090BB6
:1017EB000000000000070002030507090A000000C3
:1017FB000000070001030507080A000000000007AE
:10180B000002040607090B00000000000700020499
:10181B000507090A0000000000070002030507087E
:10182B000A0000000000070001030506080A00007B
:10183B00000000070001030507090B000000000072
:10184B00070001030507080B000000000009000258
:10185B000304060708090B00000008000103040637
:10186B0007090A00000000070001040506090A0029
:10187B0000000000070002040607090A0000000030
:10188B000005000103070800000000000000050030
:10189B000205070900000000000000050002040714
:1018AB00090000000000000005000305070A000006
:1018BB00000000000005000204060A000000000002
:1018CB000000070001040507080A000000000008DB
:1018DB00000103040607090A0000000006000204C9
:1018EB0006080A0000000000000700020406080AB0
:1018FB000B000000000003000307000000000000C5
:10190B0000000003000407000000000000000000BE
:10191B002020202020202020416C67657269616E99
:10192B002020202020202020204172616269616EDE
:10193B0020202020202042616C696E657369616EE6
:10194B002020202020426C756573206D616A6F72B8
:10195B002020202020426C756573206D696E6F729C
:10196B002020202020202042797A616E74696E65D8
:10197B00202020202020204368726F6D61746963E2
:10198B002020202020202020446961746F6E696321
:10199B0020446F75626C65204861726D6F6E696370
:1019AB0020202020202020456E69676D61746963BB
:1019BB002020202020202020456779707469616EDB
:1019CB002020202020202048696E64757374616E7E
:1019DB002048756E67617269616E206D616A6F7206
:1019EB002048756E67617269616E206D696E6F72EA
:1019FB004A6170616E3A2068697261796F736869C8
:101A0B004A6170616E3A697761746F796F73686957
:101A1B004A6170616E3A6B756D6F69796F73686946
:101A2B004A6170616E3A2020202020696E73656ECA
:101A3B004A6170616E3A2020202020796F73656EA9
:101A4B004A6170616E3A2020726974737573656EAA
:101A5B004A6170616E3A2020202072796F73656E37
:101A6B002020206D616A6F72204C6F637269616E0A
:101A7B002020207375706572204C6F637269616EE4
:101A8B00202020204C796469616E206D696E6F7225
:101A9B004D696E6F72206861726D6F6E6963203174
:101AAB004D696E6F72206861726D6F6E6963203263
:101ABB004D696E6F72206861726D6F6E6963203352
:101ACB004D696E6F72206861726D6F6E6963203441
:101ADB004D696E6F72206861726D6F6E6963203530
:101AEB004D696E6F72206861726D6F6E696320361F
:101AFB004D696E6F72206861726D6F6E696320370E
:101B0B002020204D696E6F72206D656C6F64696368
:101B1B004D6F64653A20496F6E69616E2F4D616A36
:101B2B004D6F64653A2020202020446F7269616EEE
:101B3B004D6F64653A202020506872796769616E39
:0E1B4B004D6F64653A20202020204C7964699B
:101B5900616E4D6F64653A204D69786F6C7964697F
:101B6900616E4D6F64653A41656F6C69616E2F4DA9
:101B7900696E4D6F64653A202020204C6F6372694D
:101B8900616E4E6561706F6C6974616E206D616A1A
:101B99006F724E6561706F6C6974616E206D696EEC
:101BA9006F72202020202020204E696E6520546FFE
:101BB9006E65202020202020204F637461746F6E91
:101BC900696320202020202020204F7269656E74CF
:101BD900616C20202020202020204F766572746FB0
:101BE9006E65202020202020202020202050656C98
:101BF9006F6720202020202050656E7461746F6EFD
:101C090069636D616A6F722050656E7461746F6E7D
:101C190069636D696E6F722050656E7461746F6E61
:101C2900696320202020202050726F6D65746865DB
:101C390075732020202020202020205370616E6998
:101C49007368202020202053796D6D657472696353
:101C5900616C2020202020202057686F6C65746FEC
:101C69006E656C656164696E6757686F6C65746FE2
:101C79006E656D696E6F7220547269616443686F35
:101C890072646D616A6F7220547269616443686F2E
:101C9900726420202020202075736572207363618F
:101CA9006C65010000000001000000000000000058
:101CB90000000000E53F30E407121CFA121E2D2235
:101CC900121CD0121CE52220020122C20590011724
:101CD900E004120D17F0121D42C202222003012254
:101CE900C205900117E014120D17F0C203121D422C
:101CF90022E53E30E10122E53E30E01530E31730C0
:101D0900E52DE53F30E72330E11130E21830E310EB
:101D1900227401021D3A7402021D3A7403021D3A2B
:101D29007404021D3A7405021D3A7406021D3A74C0
:101D390007900117F0121D4222900117E01475F067
:101D490003A4901D4F73021D64021D74021D8402B9
:101D59001D96021DAF021DC2021DCF74019001170D
:101D6900F0121DE51220BC123918227402900117D5
:101D7900F0121DE51225101239342274039001174F
:101D8900F0121DE5E54E1235CA123636227404905A
:101D99000117F0121DE51229C7533C21533D414358
:101DA9003C14433D28227405900117F0121DE55398
:101DB9003C21533D41433D28227406900117F012FE
:101DC9001DE51228A5227407900117F0121DE5538D
:101DD9003C21533D41433C02433D2822900117E0F9
:101DE900B40106901155021E22B4020690115F0239
:101DF9001E22B40306901169021E22B40406901132
:101E090073021E22B4050690117D021E22B4060635
:101E1900901187021E2290119105A29000007B0A61
:101E29001204B722900117E01475F003A4901E3A2A
:101E390073021E5D02227502344D0228F6023B2010
:101E4900022870023968900FDF05A29000097B040F
:101E59001204B722121E70121E88121EA01221AC83
:101E69001237331236D32220020122C205900120F3
:101E7900E004120D9CF0900120F0C202D23422201D
:101E8900030122C205900120E014120D9CF090017B
:101E990020F0C203D23422900120121EAD900120FD
:101EA90012200122E0B42B06901633021FED50F8E0
:101EB9001475F006A4901EC273901393021FBB9071
:0E1EC90013A3021FBB9013B3021FBB9013C3E1
:101ED700021FBB9013D3021FBB9013E3021FBB90DB
:101EE70013F3021FBB901403021FBB901413021FAE
:101EF700BB901423021FBB901433021FBB901443E3
:101F0700021FBB901453021FBB901463021FBB90A8
:101F17001473021FBB901483021FBB901493021FFC
:101F2700BB9014A3021FBB9014B3021FBB9014C332
:101F3700021FBB9014D3021FBB9014E3021FBB9078
:101F470014F3021FBB901503021FBB901513021F4A
:101F5700BB901523021FBB901533021FBB9015437F
:101F6700021FBB901553021FBB901563021FBB9046
:101F77001573021FBB901583021FBB901593021F99
:101F8700BB9015A3021FBB9015B3021FBB9015C3CF
:101F9700021FBB9015D3021FBB9015E3021FBB9016
:101FA70015F3021FBB901603021FBB901613021FE7
:101FB700BB90162305A29000107B101204B71222C3
:101FC7000090000D7450F02205A29000107B1012B3
:101FD70004B7900FDF05A290000A7B031204B790A5
:101FE700000D7450F02205A29000107B101204B768
:101FF70012220090000D7455F022E0B42B0302204A
:102007001150FB90000E1206E322C3942A90000E93
:102017001206E32220340122C23412203D12223A52
:102027001220BC123918900120E0F56B90015A126A
:102037003CC5E56BF022900120E0B42B030220861B
:1020470050FB1475F005A4FB9012C193FC0BEB93A6
:10205700254EFD0BEB93254EFE0BEB93254EFF0B09
:10206700EB93254E90003CF090003BEFF090003A48
:10207700EEF0900039EDF0900038ECF0F5602212A8
:102087003EAE90027FE0FBA3E0254EFCA3E0254E89
:10209700FDA3E0254EFEA3E0254E90003CF0900006
:1020A7003BEEF090003AEDF0900039ECF0900038FC
:1020B700EBF0F56022533C21533D41E560B400014C
:1020C70022B40108900039E012216322B4020F9074
:1020D7000039E012216390003AE012216322B40331
:1020E70016900039E012216390003AE012216390C4
:1020F700003BE012216322900039E0122163900037
:102107003AE012216390003BE012216390003CE02B
:1021170012216322900117E0B40507300C04123C2A
:102127002F22900039E025532555120BF7120B3754
:1021370090003AE025532555120BF7120B409000FB
:102147003BE025532555120BF7120B4990003CE055
:1021570025532555120BF7120B522222F9E5637509
:10216700F00CA4C3C999120E7375F004A4902178DA
:1021770073433C0222433C0422433C0822433C1065
:1021870022433C4022433C8022433D0222433D04FC
:1021970022433D0822433D1022433D2022433D80F8
:1021A70022433D0022900117E0B401030221B72228
:1021B700E53E30E10122E53E30E20AE53F30E01F2F
:1021C700C210C21122201016D210900142123CC533
:1021D700E004120D63F0900124F012222D22222038
:1021E7001116D211900142123CC5E014120D63F092
:1021F700900124F012222D2222900124E01475F080
:1022070006A490220D7390119B0222229011A00226
:1022170022229011A50222229011AA05A29000085D
:102227007B051204B72212203D12223A1220BC125B
:10223700391822900124E0B4010122B40208900069
:0E22470039E0240CF022B4030F900039E0249B
:102255000CF090003AE0240CF022900039E0240CB8
:10226500F090003AE0240CF090003BE0240CF022C2
:102275001222921222AA1222C2900FDF05A290000A
:10228500087B051204B71237331236D32220020118
:1022950022C205900121E004120DAFF0900121F05A
:1022A500C202D2352220030122C205900121E01489
:1022B500120DAFF0900121F0C203D2352290012119
:1022C5001222D2121E4F90012112245222E0B4395B
:1022D50007901C9B121FED2250F7B42B030222E737
:1022E500400BC3942B75F006A49023F7731475F077
:1022F50006A49022FB7390191B02244E90192B0201
:10230500244E90193B02244E90194B02244E9019ED
:102315005B02244E90196B02244E90197B02244EC9
:1023250090198B02244E90199B02244E9019AB02F2
:10233500244E9019BB02244E9019CB02244E9019BD
:10234500DB02244E9019EB02244E9019FB02244E19
:10235500901A0B02244E901A1B02244E901A2B023F
:10236500244E901A3B02244E901A4B02244E901A8A
:102375005B02244E901A6B02244E901A7B02244E67
:10238500901A8B02244E901A9B02244E901AAB028F
:10239500244E901ABB02244E901ACB02244E901A5A
:1023A500DB02244E901AEB02244E901AFB02244EB7
:1023B500901B0B02244E901B1B02244E901B2B02DC
:1023C500244E901B3B02244E901B4B02244E901B27
:1023D5005B02244E901B6B02244E901B7B02244E05
:1023E500901B8B02244E901B9B02244E901BAB022C
:1023F500244E901BBB02244E901BCB02244E901BF7
:10240500DB02244E901BEB02244E901BFB02244E54
:10241500901C0B02244E901C1B02244E901C2B0278
:10242500244E901C3B02244E901C4B02244E901CC3
:102435005B02244E901C6B02244E901C7B02244EA2
:10244500901C8B02244E901C9B121FCF22E0B439A6
:102455000302246250FB90000E1206E322C3943857
:1024650090000E1206E32220350122C23512248B7C
:10247500122510123934900121E0F56B9001A2125A
:102485003CC5E56BF022900121E0B4390D123EC840
:1024950090003DE0C3954EF5612250F11224E2050E
:1024A500A290003DF0F5611224D122B4390D123EFF
:1024B500E290004AE0C3954EF5622250F11224E203
:1024C50005A290004AF0F5621224D122A305A20BC1
:1024D500EB9305A2254EF0A305A2DAF322B413036C
:1024E5000224EA5006901643022507B42603022467
:1024F500F8500990173AC39413022507901831C371
:1025050094261475F00DA4FB93FA22533C21533DF8
:102515004190003DE0FA700122A3E005A21221637B
:1025250005A2DAF522120A181209BCB437030225EE
:1025350043500BD294533CFE533DFEC20922433C0B
:102545000130090122D2091546E54660012212270C
:10255500FA1225D59001EA123CC5E0F546C294432E
:102565003D01E545B54709754500123398022577C4
:1025750050F51225A1122580054522E02553254950
:102585002556256712258D22F9900117E0B405041B
:10259500300C0122E9120BF7120B5B22E54CB40556
:1025A500041225BE221225AE229000B7E5822545EC
:1025B500F582E5833400F58322E547120CA3F54542
:0E25C5009000B7E5822545F582E5833400F5E8
:1025D3008322900172123CC5E0B401041225EA2261
:1025E300B4020312261522E54CB401079000B7127A
:1025F300265B22B402079000B712268B22B4030491
:102603001226F222B40404122709229000B71226DC
:102613005B22E54CB401079000B712273822B402BD
:10262300079000B712276822B403041227CF22B4FD
:1026330004041227E6229000B712273822E56070BF
:10264300057E01790122FEF922E560B402057E02CE
:1026530079022240F9FEF922122640AB4B0B7A0095
:1026630005A290003912267FEEF9EA240CFA9000B5
:1026730039DBF2E54B048EF0A4F54722E02AA305EB
:10268300A2F0A305A2D9F522122640AB4BEB75F0BD
:102693000CA4FA0B05A2900038123CF61226BAEEEF
:1026A300F9EAC3940CFA900038123CF6DBEEE54BE2
:1026B300048EF0A4F54722E02AFF123CE805A2EFBE
:1026C300F0A305A2D9F12212264C19AB4BEB75F0FE
:1026D3000CA4FA0B05A2900038123CF61226BAEEAF
:1026E300F9EAC3940CFA900038123CF6DBEE229020
:1026F30000B712265B05A21226CAE54775F002A4AD
:10270300C39402F547229000B712265B05A2122656
:102713008BE54775F002A4F54722E56170057E015C
:10272300790122FEF922E561B402057E02790222D3
:1027330040F9FEF92212271DAB4B0B7A0005A2903C
:10274300003E12275CEEF9EA240CFA90003EDBF21D
:10275300E54B048EF0A4F54722E02AA305A2F0A3DB
:1027630005A2D9F52212271DAB4BEB75F00CA4FA89
:102773000B05A290003D123CF6122797EEF9EAC32F
:10278300940CFA90003D123CF6DBEEE54B048EF020
:10279300A4F54722E02AFF123CE805A2EFF0A305C7
:1027A300A2D9F12212272919AB4BEB75F00CA4FA2D
:1027B3000B05A290003D123CF6122797EEF9EAC3EF
:1027C300940CFA90003D123CF6DBEE229000B71217
:1027D300273805A21227A7E54775F002A4C3940280
:1027E300F547229000B712273805A2122768E5475C
:1027F30075F002A4F54722122863900127E0B40183
:10280300149001D2123CC5E0F54CE54A120E60F576
:102813004B75490022B402189001D2123CC5E0F571
:102823004C754B00E54A120E4D75F00CA4F5492288
:10283300B4030EE54A120DEEF54C754B00754900D5
:1028430022B4040EE54A120DEEF54C754B017549A1
:102853000022E54A120DEEF54C754B027549002234
:10286300120A0C120A4A75F00C84F54A22122877D0
:1028730012288E2220020122900127E004120E3A30
:10288300F0900127F01228A5C20222200301229012
:102893000127E014120E3AF0900127F01228A5C286
:1028A3000322533C21533D419011B905A2900009E5
:1028B3007B071204B71228BC22900127E0120E3ABC
:1028C300F01475F006A49028CD739011C00228EB84
:1028D3009011D00228EB9011E00228EB9011F00246
:1028E30028EB9012000228EB05A29000107B101237
:1028F30004B72212298E122903122ECE1236D322A6
:10290300E53E30E10412294F2212291022E53E3020
:10291300E222E53F30E005C210C21122201014D29A
:1029230010900129E004120F3CF01241471229C70D
:102933001232EC22201114D211900129E014120F4B
:0E2943003CF01241471229C71232EC22E53E49
:1029510030E222E53F30E005C210C21122201014FE
:10296100D21090011AE004120D89F0122BA4122941
:10297100C71232EC22201114D21190011AE0141264
:102981000D89F0122BA41229C71232EC22E53E2048
:10299100E10122E53F30E60AE53E30E417C214C208
:1029A100152220140ED214900119E014120D76F0A4
:1029B1001229C72220150ED215900119E004120D1B
:1029C10076F01229C722900119E0B40124122BBB21
:1029D10090101305A29000107B011204B790012AF8
:1029E100122D0C90101405A29000147B011204B753
:1029F10022B40221122BBB90101305A29000157B6B
:102A0100011204B7122D3D90101405A290001A7BFB
:102A1100011204B722B40328122BBB90101305A294
:102A210090001B7B011204B790015A123CC5E012C1
:102A31002D6D90101405A290001F7B011204B72286
:102A4100B40404122BEF22B40904122C0622B40A96
:102A510004122C4422900172123CC5E0B40304120A
:102A61002B012250FA122A6A22900119E0B405279B
:102A7100122C5B90101305A29000107B011204B779
:102A810090018A122D2C90101405A29000147B0144
:102A91001204B7122E5722B40621122C5B90101388
:102AA10005A290001B7B011204B7122E579010143F
:102AB10005A290001F7B011204B722B40721122C3A
:102AC1008590101305A29000137B011204B7122EFA
:102AD1007990101405A29000187B011204B72212FC
:102AE1002C8590101305A290001C7B011204B79055
:102AF100101405A290001F7B011204B7122EAF2201
:102B0100900119E0B40524122CAC90101305A29089
:102B110000107B011204B7900202122D2C901014A8
:102B210005A29000147B011204B722B40627122CCF
:102B3100AC90101305A290001B7B011204B7900208
:102B410032123CC5122DAC90101405A290001F7BCF
:102B5100011204B722B40724122CDC90101305A231
:102B61009000107B011204B790021A122D2C9010C4
:102B71001405A29000147B011204B722122CDC90E0
:102B8100101305A290001B7B011204B790024A1298
:102B91003CC5122D9390101405A290001F7B0112C9
:102BA10004B72290011AE09000061206E322900178
:102BB10029E0142441900005F022122BAF122BA41E
:102BC10090107505A29000097B071204B7901015AB
:102BD10005A29000107B101204B790012A122D0C4F
:102BE100122D3D90015A123CC5E0122D6D22122B7F
:102BF100AF122BA490107C05A29000097B07120450
:102C0100B7122DD222122BAF122BA490109105A234
:102C11009000097B071204B7900FDF05A290001006
:102C21007B0C1204B790101305A290001C7B0112BB
:102C310004B7122E0290101405A290001F7B0112FE
:102C410004B722122BAF122BA490109805A290006A
:102C5100097B071204B7122E0D22122BAF122BA4DF
:102C610090108305A29000097B071204B7901025EC
:102C710005A29000107B101204B790018A122D2C2E
:102C8100122E2E22122BAF122BA490108305A2908C
:102C910000097B071204B790103505A29000107B44
:102CA100101204B7122E79122EAF22122BAF122B53
:102CB100A490108A05A29000097B071204B7901016
:0E2CC1004505A29000107B101204B79002028D
:102CCF00122D2C900232123CC5122DAC22122BAFBA
:102CDF00122BA490108A05A29000097B071204B74B
:102CEF0090105505A29000107B101204B790021A95
:102CFF00122D2C90024A123CC5122D9322123CC564
:102D0F00E075F00C84FEE5F012369B05A2900011E1
:102D1F007B021204B7EE9000131206DF22123CC59D
:102D2F00E09000121206E3900011742BF022900134
:102D3F0042123CC5E01475F006A4902D4D7390110E
:102D4F009B022D629011A0022D629011A5022D629F
:102D5F009011AA05A29000167B041204B722E0B4CA
:102D6F002B03022D8350FB90001D1206E390001CD5
:102D7F007450F022C3942A90001D1206E390001C99
:102D8F007455F022E06003022DAD90001C743DF0ED
:102D9F0090001D7462F090001E7469F022E0B43947
:102DAF0003022DC250FB90001D1206E390001C740D
:102DBF0050F022C3943890001D1206E390001C744B
:102DCF0055F022900172123CC5E01475F006A490E4
:102DDF002DE2739010CF022DF79010DF022DF79098
:102DEF0010EF022DF79010FF05A29000107B10122C
:102DFF0004B72290027AE090001D1206E32290029F
:102E0F007BE01475F006A4902E1A7390112F022EEA
:102E1F002390113F05A29000107B101204B722904F
:102E2F000172123CC5E0B4010E90110F05A2900083
:102E3F00167B051204B722B4020D90111405A2904F
:102E4F0000167B051204B722900172123CC5E0B444
:102E5F00010A90015A123CC5122D6D22B4020A903C
:102E6F0001A2123CC5E0122DAC229001D2123CC53A
:102E7F00E01475F006A4902E8973901119022EA4F8
:102E8F0090111D022EA4901121022EA49011250243
:102E9F002EA490112905A29000147B041204B722CE
:102EAF009001EA123CC5E0B4010E90112D05A290DD
:102EBF00001D7B021204B72290001D1206E3229020
:102ECF000119E0B40107122F78122F9422B40207D0
:102EDF00122FB0122FC922B40307122FE2122FFBA9
:102EEF0022B4040712301412302D22B40907123005
:102EFF004612305922B40A0712306C12307F2290DA
:102F0F000172123CC5E0B40304122F4C2250FA1286
:102F1F002F2222900119E0B405071230921230AE21
:102F2F0022B406041230CA22B407071231461231F6
:102F3F005F22B408071231781231902222900119C2
:102F4F00E0B405071231A81231C422B406071231BA
:102F5F00E01231F922B4070712321212322E22B4C4
:102F6F00080612324A123263222002012290012AED
:102F7F00123CC5E004120EAAF090012A122D0C1279
:102F8F0032ECC202222003012290012A123CC5E03A
:102F9F0014120EAAF090012A122D0C1232ECC20359
:102FAF002220020122900142123CC5E004120D635F
:102FBF00F0122D3D1232ECC20222200301229001A9
:102FCF0042123CC5E014120D63F0122D3D1232EC8B
:102FDF00C203222002012290015A123CC5E00412C2
:102FEF000D9CF0122D6D1232ECC202222003012231
:102FFF0090015A123CC5E014120D9CF0122D6D1267
:10300F0032ECC2032220020122900172123CC5E071
:10301F0004120DDBF0122DD21232ECC20222200369
:10302F000122900172123CC5E014120DDBF0122D3B
:0E303F00D21232ECC203222002012290027A49
:10304D00E004120EBAF0122E02C202222003012257
:10305D0090027AE014120EBAF0122E02C203222050
:10306D0002012290027BE004120ECDF0122E0DC251
:10307D0002222003012290027BE014120ECDF012E9
:10308D002E0DC203222002012290018A123CC5E0BE
:10309D0004120EAAF090018A122D2C1232ECC202EB
:1030AD00222003012290018A123CC5E014120EAABF
:1030BD00F090018A122D2C1232ECC2032290017273
:1030CD00123CC5E0B401071230E21230FB2212317E
:1030DD001412312D222002012290015A123CC5E01A
:1030ED0004120D9CF0122D6D1232ECC2022220033F
:1030FD00012290015A123CC5E014120D9CF0122DC4
:10310D006D1232ECC20322200201229001A2123C68
:10311D00C5E004120DAFF0122DAC1232ECC202223A
:10312D00200301229001A2123CC5E014120DAFF054
:10313D00122DAC1232ECC20322200201229001D2D8
:10314D00123CC5E004120DEEF0122E791232ECC2D3
:10315D000222200301229001D2123CC5E014120D6F
:10316D00EEF0122E791232ECC203222002012290CF
:10317D0001EA123CC5E004120E01F0F546122EAF25
:10318D00C20222200301229001EA123CC5E0141272
:10319D000E01F0F546122EAFC2032220020122903D
:1031AD000202123CC5E004120EAAF0900202122D8A
:1031BD002C1232ECC2022220030122900202123C98
:1031CD00C5E014120EAAF0900202122D2C1232EC50
:1031DD00C2032220020122900232123CC5E00412E9
:1031ED000DAFF0122DAC1232ECC2022220030122DF
:1031FD00900232123CC5E014120DAFF0122DAC123C
:10320D0032ECC203222002012290021A123CC5E0C8
:10321D0004120EAAF090021A122D2C1232ECC202D8
:10322D00222003012290021A123CC5E014120EAAAC
:10323D00F090021A122D2C1232ECC2032220020140
:10324D002290024A123CC5E004120DC2F0122D93D9
:10325D001232ECC202222003012290024A123CC516
:10326D00E014120DC2F0122D931232ECC203229013
:10327D00027BE0B4010412328B221232C0221209F9
:10328D00F4120A4AB55D0122533DBFF55D120EF3EE
:10329D0090011AF01232EC900117E0B401041220E3
:1032AD00BC22B4020412251022B40406122BA4125F
:1032BD0029C7221209F41209BCB437030232D450C3
:1032CD0006533DBFC20D22433D40200D11D20D903E
:1032DD00011AE004120F0E90011AF01232A122D23F
:1032ED000A90012A123CC5E075F00C8485F04E75EC
:1032FD00F00CA4F55590015A123CC5E0900120F058
:10330D00900142123CC5E0900124F012203D1222A2
:10331D003A12391890018A123CC5E0F55690020216
:10332D00123CC5E0F55790021A123CC5E0F55890D5
:10333D000172123CC5E0900122F0123398B40304DF
:10334D0012336F2250FA1233572220330302336E99
:10335D009001A2123CC5E0900121F012248B12398C
:10336D00342290024A123CC5E0600E123386900260
:10337D004A123CC5E01224B022900232123CC5E044
:10338D00900121F012248B12393422900122E0B4E5
:10339D000103C23322B40202D23322900122E0B4DF
:1033AD0003041233DB22B404031233BA22120A18B7
:0E33BD001209BCB437030233CE5006533CFE57
:1033CB00C20922433C0130090122D2091233DB220C
:1033DB00120A0C120A4A120EA1B55A10200A4B22DD
:1033EB00F55A85575990003D1234192250F2F55A6F
:1033FB0085585990024A123CC5E0600990004AE595
:10340B005A1234192290003DE55A1234192275F0E4
:10341B000C8485F06B75F00CA4FAE0F9A3E0C3956E
:10342B004EB56B03023435D9F322C20AF54D254E46
:10343B002A25592553256712258DC294433D01D268
:10344B003622E53E20E10412346C221234C21234CF
:10345B00CB1235A7E54E1235CA123636C202C2035D
:10346B0022900117E0B4030302347722E53E30E4E7
:10347B000AE53F30E623C212C2132220121AD212DF
:10348B00E566F56B04120E91F566B56B0302349D80
:10349B00D20A1234C21236362220131AD213E56620
:1034AB00F56B14120E91F566B56B030234BBD20AA1
:1034BB001234C212363622E56675F00CA4F567227B
:1034CB00E53E20E005740002353620E2057401026A
:1034DB00353620E3057402023536E53F20E50574E9
:1034EB000602353620E005740302353620E10574FB
:1034FB000402353620E305740502353620E20574E7
:10350B000702353620E605740802353620E70574C8
:10351B0009023536E53E20E405740A02353620E50E
:10352B0005740B023536E54EC22E22202E30D22EDC
:10353B00854E4FF54E12356A123576900125E54EC4
:10354B00F0A3F0F990012A123CC5E075F00C8475DC
:10355B00F00CA4254EF01225D5D20A1232EC229093
:10356B00003874041235811239182290003DE01294
:10357B00359412393422FA700122A3E0FC254EC394
:10358B00954F120E83F0DAF222FA700122A3E0FCBF
:10359B00254EC3954F120E83F0DAF222120A001257
:1035AB000A4AB43C030235B6400122F553B5540127
:1035BB0022F55475F00C84F55C85F05BD20A22532E
:1035CB003C21533D41120E7375F007A49035DB730C
:1035DB00533D41433C0222533D41433C0422533D66
:1035EB0041433C0822533D41433C1022533D414350
:1035FB003C4022533D41433C8022533C21433D02FE
:10360B0022533C21433D0422533C21433D0822538A
:10361B003C21433D1022533C21433D2022533C216E
:10362B00433D8022533C21533D4122900FDF05A2A5
:10363B0090000A7B041204B7E54E12369B05A2904C
:10364B00000D7B021204B7E56690000F1206DF90A7
:10365B0011AF05A29000107B0A1204B7900FDF0583
:10366B00A290001A7B031204B7E55490001E1206B9
:10367B00E390001D742BF022E55B12369B05A290A4
:10368B00001D7B021204B7E55C90001F1206DF22BF
:10369B0075F004A49036A3739012A9229012AB225A
:1036AB009012AD229012AF229012B1229012B3223F
:1036BB009012B5229012B7229012B9229012BB220F
:1036CB009012BD229012BF22900117E0B4010302A9
:1036DB0036EAB402030236EAB404030236EA22E500
:1036EB003E30E10122E53E30E40AE53F30E616C20A
:1036FB0012C2132220120DD212E56304120E91F5A1
:10370B00631237212220130DD213E56314120E918D
:10371B00F56312372122900117E0B401041220BC8B
:10372B0022B4020312251022E53E20E101221237BA
:0E373B005E12377212378612379A1237AE12AC
:1037490037C21237D61237EA1237FE123812123838
:103759002612383A22E53E30E003C20F22200F0834
:10376900D20F90005712384E22E53E30E203C216BE
:1037790022201608D21690005812384E22E53E3003
:10378900E303C21722201708D21790005912384EA6
:1037990022E53F30E003C21822201808D218900011
:1037A9005A12384E22E53F30E103C2192220190886
:1037B900D21990005B12384E22E53F30E303C21A5A
:1037C90022201A08D21A90005C12384E22E53F30A6
:1037D900E503C21B22201B08D21B90005D12384E44
:1037E90022E53F30E203C21C22201C08D21C9000B3
:1037F9005E12384E22E53F30E603C21D22201D0825
:10380900D21D90005F12384E22E53F30E703C21EF9
:1038190022201E08D21E90006012384E22E53E304A
:10382900E403C21F22201F08D21F90006112384EE4
:1038390022E53E30E503C22022202008D220900054
:103849006212384E2205A2900117E0B4010905A2BF
:10385900123C8212386F22B4020B05A2123CA61246
:103869003C821238BE22E020E01DE560B4040F0559
:10387900A27B0490005612390D05A202388950EF37
:10388900E0D2E0F0023893C2E0F07C007B007A30AD
:1038990090005705A290003905A2E030E0080BEC32
:1038A90005A2F0A305A2A30CDAF0900038EBF0F51D
:1038B900601220BC22E020E01DE561B40C0F05A2D6
:1038C9007B0C90008612390D05A20238D850EFE022
:1038D900D2E0F00238E2C2E0F07C007B007A30905E
:1038E900008705A290003E05A2E030E0080BEC0538
:1038F900A2F0A305A2A30CDAF090003DEBF0F5616C
:1039090012251022A3E030E0FBDBF9C2E0F022121D
:103919003950900038E0FBA3E004FA05A290005664
:10392900A3DAFD7401F005A2DBED2212395C9000E7
:103939003DE0FBA3E004FA05A2900086A3DAFD743A
:1039490001F005A2DBED2290005774007930F0A355
:10395900D9FC2290008774007930F0A3D9FC221297
:103969003978123A47123A9D1239B2123AD922E5F8
:103979003E20E10122E53F30E60AE53E30E414C28B
:1039890014C2152220140BD21490011CE014120F3A
:1039990029F02220150BD21590011CE004120F29E1
:1039A900F02290000E1206E32290011CE0B40101FE
:1039B90022B402071239D51239E822B403071239A1
:1039C900FB123A0E22123A21123A34222002012223
:1039D90090011DE004120D50F01239ABC2022220F1
:1039E90003012290011DE014120D50F01239ABC2EF
:1039F90003222002012290011EE004120D50F01250
:103A090039ABC202222003012290011EE014120DDB
:103A190050F01239ABC2032220020122900129E0A1
:103A290004120F3CF0123A91C202222003012290A3
:103A39000129E014120F3CF0123A91C203229001BD
:103A49001CE0B4010E90121005A29000057B0B1228
:103A590004B722B4020E90121B123ACE90011DE057
:103A69001239AB22B4030E901226123ACE90011EDF
:103A7900E01239AB22901231123ACE123A919000EB
:103A89000E7420F0123A9122900129E014244190F9
:103A9900000FF022900035E060012290123C05A24F
:103AA9009000107B101204B72290124C05A29000CE
:0E3AB900107B101204B722900FCF05A29000D0
:103AC700107B101204B72205A29000057B0912048F
:103AD700B722E53E30E003C20B22200B1BD20B12AC
:103AE7003AC0120203C2AF123B00D2AF12036612F2
:103AF7003AB29000357404F02290011CE0B401043E
:103B0700123E4B22B40204123E7122B40304123E49
:103B17008422124113123E4B22123B2A123B5D12A2
:103B27003BB122E53E20E10122E53F30E60AE53ED2
:103B370030E414C214C2152220140BD21490011FB2
:103B4700E014120EE0F02220150BD21590011FE0B1
:103B570004120EE0F02290011FE0B4011190125CF4
:103B670005A29000067B0A1204B7123BE6229012C8
:103B77006605A29000067B0A1204B7123B862290C4
:103B87000128E0B4010E90127005A29000107B107E
:103B97001204B7221414244190001FF090128005DC
:103BA700A29000107B0F1204B72290011FE0B4010E
:103BB70007123BC6123BD622123C62123C722220ED
:103BC700020122900118E004120D2AF0C2022220FD
:103BD700030122900118E014120D2AF0C20322906B
:103BE700129005A29000107B0D1204B7900118E007
:103BF700B4011090114F05A290001D7B031204B76A
:103C0700C20C22141490001E1206DF90129D05A20A
:103C170090001D7B011204B790129F05A290001F10
:103C27007B011204B7D20C22900118E0141475F02E
:103C37000CA4F565120BF7120B37E565120BF7129B
:103C47000B40E565120BF7120B49E565120BF712EE
:103C57000B52E565120BF7120B5B22200201229033
:103C67000128E004120D3DF0C20222200301229038
:103C77000128E014120D3DF0C20322E56375F00C34
:103C8700A48582328583337534007535007832F523
:103C9700367537007936120229868208868322858F
:103CA7008232858333753400753500783275363046
:103CB7007537007936120229868208868322858223
:103CC70032858333753400753500783290011AE0F8
:103CD70014F53675370079361202298682088683ED
:103CE70022C3E5829401F582E5839400F58322E5FA
:103CF7008229F582E5833400F58322858232858324
:103D070033753400753500783290011DE01475F075
:103D170005A4023D338582328583337534007535BA
:103D270000783290011EE01475F00DA4F536753752
:103D37000079361202298682088683228582328597
:103D47008333753400753500783275F005023D68A8
:103D5700858232858333753400753500783275F086
:103D67000DA4F53675370079361202298682088642
:103D770083227532557533017534007535007832F5
:103D870014F5367537007936120244868208868321
:103D970022901CAB05A29000007E1005A27F0512A1
:103DA7003DC8901CAB05A2DEF22290003D05A29013
:103DB70000A07E1005A2790D123DFF90003DDEF6B2
:103DC7002274009343D20205A2F0A375D25275D292
:103DD700A2E5D220E0FB53D2FD05A2A3DFE32290A8
:103DE700003D05A2901CB07B0DE493A305A2F0A3B0
:103DF70005A2DBF5123DB122E0A343D20205A2F0F2
:103E0700A375D25275D2A2E5D220E0FB53D2FD05AD
:103E1700A2D9E52243D202438E20E0A353D2FD5319
:103E27008EDF05A2F0A305A2D9EA2243D202438E70
:0E3E370020E0254EA353D2FD538EDF05A2F0EE
:103E4500A305A2D9E822790A90012005A290024093
:103E550005A2123DFF22900125E54EF0A3E54FF0A6
:103E650022900125E0F54EA3E0F54F22900038059C
:103E7500A2900000123D0205A27905123DFF229095
:103E8500003D05A29000A0123D1C05A2790D123D32
:103E9500FF22C2AF790A90024005A290012005A237
:103EA500123E1B123E66D2AF22C2AF900000C394F1
:103EB5002B123D4305A290027F05A27905123E1BF8
:103EC500D2AF22C2AF9000A0C39439123D5705A2CC
:103ED50090003D05A2790D123E32D2AF22C2AF90BD
:103EE50000A0C39439123D5705A290004A05A27956
:103EF5000D123E32D2AF22E53E30E10122753C1073
:103F0500900FAF05A29000007B101204B7900FBF71
:103F150005A29000107B101204B7E53E30E1FBE5E9
:103F25003F30E00630E632023F24E53F30E0FB1249
:103F35000203120203900FCF05A29000107B10120E
:103F450004B7120203120203C2AF123D98123DE6F6
:103F5500123F6A123FAAD2AF22E53F30E6FB1202BA
:103F650003120203229001207416F09001217401BE
:103F7500F09001227401F09001237401F090012466
:103F85007401F09001257400F09001267400F09002
:103F950001277401F09001287401F0900129740142
:103FA500F0123E4B2290027A7418F090027B740155
:103FB500F090012A740012403E90018A740012406C
:103FC5003E900202740012403E90021A74001240A4
:103FD5003E900142740112403E90015A741B1240FA
:103FE5003E900172740112403E9001A2742F12405E
:103FF5003E9001BA741B12403E9001D274031240E8
:104005003E9001EA740112403E900232743812402B
:104015003E90024A740012403E12402222740190E2
:104025000129F0123D7912411E900129E004F0B4F6
:104035000DF17401900129F0227B18F0A3DBFC221D
:104045001240E574A0F91240B21240FBE568F9127E
:1040550040B21240FBE569F91240B21240FB124032
:10406500E574A1F91240B21240FB1240A5124101BC
:104075001240D722E9FA1240E574A0F91240B212B3
:104085004101E568F91240B2124101E569F91240B2
:10409500B2124101EAF91240B21241011240D7228F
:1040A500D2A57808124107E933F9D8F8227808E94A
:1040B5003392A5F9124107D8F6227B80DB02800EE8
:1040C5001240E574A0F91240B212410140EE1240CF
:1040D500D722C2A500D2A4000000000000D2A5226C
:1040E500D2A500D2A4000000000000C2A500000077
:1040F500000000C2A422C2A512410722D2A5124186
:1041050007220000D2A4000000A2A5C2A4229001AB
:1041150029E0123D7912411E2205A290012A05A22D
:104125007FD81241307F7D12413022858368858298
:104135006905A2E0F9A305A21240791240BFA3DFE9
:10414500EA22900129E0123D7912416C2290012862
:10415500E0B40107900129E002416514900129F0BE
:10416500123D7912416C2205A290012A05A27FD841
:1041750012417E7F7D12417E228583688582691288
:104185004045A3E905A2F0A305A2DFED227540286D
:1041950075410475427D75430275440A90FF9C85FF
:1041A50082CA8583CB8582CC8583CD43C804D2ADB5
:0E41B500D2AF22C0E0C0D0E582C0E0E583C0FA
:1041C300E0D2D4C2D3C2CFD5404675402812030CE7
:1041D300120906120917B20E12095530360DD544CD
:1041E3000A754405D294533DFEC236D5412275412A
:1041F3000612098E120C3F120C74D542137542320B
:10420300900035E0600214F0D54305754314B20500
:0D421300D0E0F583D0E0F582D0D0D0E032CD
:00000001FF
